:0A17F60000010202030304040505CC
:1009D600E4F55DF55CF55BF55AC211C20EC210C2B4
:1009E6000F1220181207E47E187F008E0A8F0B75EF
:1009F600121875131275081875091C7510187511DB
:100A06005175141875157FEE54E07003020B1D75B1
:100A16005E00755F808E608F61C374A99FFF741836
:100A26009ECF2402CF3400FEE48F598E58F557F539
:100A360056F555F554F553F552AF59AE58AD57AC7A
:100A460056AB55AA54A953A852C3120C765026E5A4
:100A56005F2555F582E55E3554F58374CDF0E55591
:100A66002401F555E43554F554E43553F553E4358E
:100A760052F55280C4E4F555F554F553F552AF5985
:100A8600AE58AD57AC56AB55AA54A953A852C3128B
:100A96000C765031AE54AF55E5612FF582E5603ED8
:100AA600F583E0FDE55F2FF582E55E3EF583EDF02B
:100AB600EF2401F555E43EF554E43553F553E4359A
:100AC60052F55280B9855E0A855F0B74002480FF5B
:100AD600741834FFFEC3E5139FF513E5129EF51255
:100AE600C3E50D9FF50DE50C9EF50CC3E50F9FF5CF
:100AF6000FE50E9EF50EC3E5099FF509E5089EF57F
:100B060008C3E5119FF511E5109EF510C3E5159F85
:100B1600F515E5149EF514D2E843D82090E668E072
:100B26004409F090E65CE0443DF0D2AFD288D28A28
:100B3600C2A8C2AA43E808D2FB90E680E020E105FD
:100B4600D212121DE490E680E054F7F0538EF8C2FC
:100B560011300F051203A4C20F301129122164505F
:100B660024C211121F64200E1690E682E030E704BC
:100B7600E020E1EF90E682E030E604E020E0E412D7
:0A0B86001E1312216612102080C712
:1003A40090E6B9E070030204551470030204D224E9
:1003B400FE700302055524FB700302044F147003FE
:1003C400020449146073146076240560030205B4C2
:1003D40012216840030205C090E6BBE024FE6022BF
:1003E40014603324FD601114602224067048E50A69
:1003F40090E6B3F0E50B8037E51290E6B3F0E51331
:10040400802DE50C90E6B3F0E50D8023E50E90E633
:10041400B3F0E50F801990E6BAE0FF121E3FAA067A
:10042400A9077B01EA494B600DEE90E6B3F0EF902B
:10043400E6B4F00205C00205B912209E0205C012FE
:10044400214F0205C0121AD50205C012208C0205E4
:10045400C012216A40030205C090E6B8E0247F6020
:100464001514601924027063A20EE43325E0FFA280
:1004740010E4334F8041E490E740F0803F90E6BCC5
:10048400E0547EFF7E00E0D394807C0040047D0134
:1004940080027D00EC4EFEED4F24F6F58274173E8B
:1004A400F583E493FF3395E0FEEF24A1FFEE34E6F9
:1004B4008F82F583E0540190E740F0E4A3F090E6E6
:1004C4008AF090E68B7402F00205C00205B912218D
:1004D4006C40030205C090E6B8E024FE60162402D6
:1004E40060030205C090E6BAE0B40105C20E02053D
:1004F400C00205B990E6BAE0705590E6BCE0547EBF
:10050400FF7E00E0D394807C0040047D0180027D66
:1005140000EC4EFEED4F24F6F58274173EF583E4AD
:1005240093FF3395E0FEEF24A1FFEE34E68F82F5CE
:1005340083E054FEF090E6BCE05480131313541F80
:10054400FFE0540F2F90E683F0E04420F0806D80AC
:100554006412216E506690E6B8E024FE601924020D
:10056400705A90E6BAE0B40104D20E804F90E6BA15
:10057400E064026047803E90E6BCE0547EFF7E006B
:10058400E0D394807C0040047D0180027D00EC4E29
:10059400FEED4F24F6F58274173EF583E493FF33A2
:1005A40095E0FEEF24A1FFEE34E68F82F583800808
:1005B400120080500790E6A0E04401F090E6A0E02D
:0305C4004480F080
:0105C7002211
:030033000215FCB7
:0415FC0053D8EF329F
:10201800758CE0758AC0E58954F04401F589758EA0
:0820280003D28CD2A9D2AF2231
:03005B00020CFB99
:0D0CFB00C0E0C083C082C0D075D000C0072B
:100D0800AF91530780EF64806003020E0353917F15
:100D1800300C03020E01E54864017043D3E53894B2
:100D2800C8E53794005003020E01902473E547F09C
:100D3800D394C8E5469400401DD3E5479408E5469A
:100D480094075012E53894B8E537940B5008752B82
:100D580001754800D202853746853847020DFBE504
:100D68004864027061C3E53894C8E5379400404888
:100D7800D3E53894C8E53794004010D3E538940893
:100D8800E53794075005752B008027D3E53894087C
:100D9800E5379407400FD3E5389468E53794105049
:100DA80004052B800DD3E5389468E5379410400886
:100DB800052B753700753800E52B652C703BF54819
:100DC800F537F5388033E548B4022ED3E538940179
:100DD800E5379400402374722534F582E43424F511
:100DE80083E538F00534052BE52BB4140675480067
:0B0DF800752B00753700753800C20C29
:0B0E0300D007D0D0D082D083D0E032E6
:1018000012010002000000401816238300000102AC
:1018100000010A0600020000004001000902350034
:1018200001010080FA0904000005FF00000007051F
:101830000102400000070582020002000705810244
:1018400040000007058602000200070508020002AA
:101850000009022E0001010080FA0904000004FFC3
:101860000000000705010240000007058202400059
:101870000007050202000200070581024000000483
:1018800003090410035100480059002D0043004390
:10189000004400160351004800590039003000414F
:0B18A0000020002000200020000000BD
:1005C8006080256C030A0101010201070000000296
:1005D800000002000A2B0B13111515110000000072
:1005E8000000003F030F02010103010700000002A1
:1005F800000002000A2B130B111511110000000056
:100608000000003F0314010101020107000000027D
:10061800000002000A2B0B13111515110000000031
:100628000000003F03140201010502070000000258
:10063800000002000A2B130B111515110000000011
:100648000000003F602425F30000000000000000C7
:100658000000000000000000000000000000000092
:100668000000000000000000000000004725EC80AA
:06067800000011CA4E0053
:1014B90090E60174CAF090E6F574FFF09025ECE02F
:1014C90090E6F3F09025EDE090E6C3F09025EEE08C
:1014D90090E6C1F09025EFE090E6C2F09025F1E0AA
:1014E90090E6C0F09025F2E090E6F4F075AF07744D
:1014F90025F59A746CF59B759DE4E4F59EFF90E6DD
:101509007BE090E67CF00FBF80F490E67174FFF009
:10151900F5B490E672E04480F043B680000000E440
:1015290090E6C4F000000090E6C5F09025F3E09045
:10153900E6C6F09025F4E090E6C7F09025F5E09036
:10154900E6C8F09025F6E090E6C9F09025F7E0901E
:10155900E6CAF09025F8E090E6CBF09025F9E09006
:0B156900E6CCF09025FAE090E6CDF013
:011574002254
:03004300021600A2
:0300530002160092
:101600000220300002207600022060000220480004
:10161000021CE100021C6D00022170000221710019
:101620000221720002217300021DB3000212250084
:101630000221740002217500021C2E00021B3400DE
:101640000221760002217100022177000221780038
:101650000221790002217A0002217B0002217C0014
:1016600002217D000221710002217100022171001E
:1016700002217E0002217F000221800002218100E0
:1016800002218200022183000221840002218500C0
:1016900002218600022187000221880002218900A0
:1016A00002218A0002218B0002218C0002218D0080
:0816B00002218E0002218F00CF
:101E130090E682E030E004E020E60B90E682E030DA
:101E2300E119E030E71590E680E04401F07F147E8D
:0C1E330000121BE890E680E054FEF02254
:101F640090E682E044C0F090E681F04387010000EF
:041F74000000002247
:101DE40030120990E680E0440AF0800790E680E033
:101DF4004408F07FDC7E05121BE890E65D74FFF07A
:0F1E040090E65FF05391EF90E680E054F7F02204
:021E3F00A907F1
:101E4100AE14AF158F828E83A3E064037017AD01CA
:101E510019ED7001228F828E83E07C002FFDEC3E14
:091E6100FEAF0580DF7E007F006A
:011E6A002255
:101BE8008E668F6790E600E054187012E56724014E
:101BF800FFE43566C313F566EF13F567801590E6C5
:101C080000E05418FFBF100BE56725E0F567E566AF
:101C180033F566E5671567AE66700215664E6005B2
:061C2800121F7880EE227D
:101F78007400F58690FDA57C05A3E582458370F97C
:011F88002236
:10067E0060A524C518244242424242424224181028
:10068E007010101010101010107C3C4242420404E6
:10069E00081020427E3C42420418040202424438B2
:1006AE00040C14242444447E04041E7E404040580E
:1006BE006402024244381C244040586442424224A0
:1006CE00187E444408081010101010103C4242428C
:1006DE002418244242423C1824424242261A020264
:1006EE00243800000000007F000000000038448223
:1006FE0082828282B2CA4C38E7424242427E4242F3
:10070E004242E7EE44442828101010101038101002
:10071E00182828243C444242E7C18342256A00003F
:10072E004224B200004224B40000412410004124AF
:10073E0011004124BB0002301040C100C108C105A8
:10074E000143000126004424C1000000004424B7E8
:10075E00000000000136004124B600604024720003
:10076E00000000000000000000000000000000007B
:10077E00000000000000000000000000000000006B
:10078E00000000000000000000000000000000005B
:10079E00000000000000000000000000000000014A
:1007AE003400014801012CFF012B0002370000022A
:1007BE00460000014500014F00024D00000232C309
:1007CE0050012A19C10AC18CC102C10B013B0001A3
:0507DE003900012F00AD
:101E6B008F629024527403F0E4A3F07A247B527DAA
:101E7B00027F41121FE19024527401F0A3E562F03E
:0B1E8B007A247B527D027F41021FE1A0
:0B211E00C2B6C2B48FB1D2B4D2B62258
:0B212900D2B6C2B48FB1D2B4D2B6223D
:041FFD00AE05AD0779
:10200100E4FCE4FBAF05122129AF061221290BBB29
:0620110060F20CBC40EC83
:0120170022A6
:101EC100AE05AD077F1512211EAF0612211E7F5FE1
:101ED10012211E7F7512211EAF0512211E7F3F1296
:0A1EE100211E7F251221290221296C
:02191E00AE0316
:10192000EDC454F0F562EE75F008A4F563BF2D0424
:101930007A0A8020BF51047A0B8019BF48047A0CC0
:101940008012BF59047A0D800BBF41047A0E8004C7
:10195000EF24D0FAE4FBEA75F00BA424C5F582E489
:101960003424F583E5822BF582E43583F583E0F9B1
:10197000E4FCE930E70DE56224032BFFE5632CFD71
:0F198000121EC1E925E0F90CBC08E70BBB0BC731
:01198F002235
:1013F600C2B77FC87E00121ABED2B77FAE12211EB8
:101406007FA012211E7F7212211E7FA112211EE4CF
:10141600FF12211E7FA212211EFF12211E7FA4127F
:10142600211E7FA812211E7F3F12211E7FAD122191
:101436001E7F8E12211E7FB012211E7F0B12211ECF
:101446007FB112211E7F3112211E7FB312211E7F12
:10145600F012211E7F8A12211E7F6412211E7F8BAD
:1014660012211E7F7812211E7F8C12211E7F64128C
:10147600211E7FBB12211E7F3A12211E7FBE122122
:101486001E7F3E12211E7F8712211E7F0612211EFD
:101496007F8112211E7F9112211E7F8212211E7FC3
:1014A6005012211E7F8312211E7F7D12211E7FAFC7
:0314B60002211EF2
:101575001213F6E4FDFF121FFD7B037D017F51125F
:10158500191E7B047D017F4812191E7B057D017F95
:101595005912191E7B067D017F3912191E7B077DA5
:1015A500017F3012191E7B087D017F4112191E7BB8
:1015B500027D027F3112191E7B037D027F381219CD
:1015C5001E7B047D027F2D12191E7B057D027F3057
:1015D50012191E7B067D027F3512191E7B077D02BF
:1015E5007F2D12191E7B087D027F3112191E7B0982
:0715F5007D027F3402191E84
:1007E40090E600E054E74410F000000000000090A0
:1007F400E61074A0F000000090E60B7401F090E69F
:100804001274E0F0000000E490E613F000000090A1
:10081400E61474E2F000000090E61574A0F0000005
:100824000090E6D27402F090E6047480F0000000B8
:100834007402F00000007406F00000007408F00078
:100844000000E4F00000001214B990E6187408F0F7
:1008540000000090E619F000000090E61AF0000095
:100864000090E61BF0000000E490E671F075B47FA0
:1008740075A07F90E672F075B6FF75B1FF90E670D3
:10088400F075B2FF75B5FFC28CD2B012215F90E64D
:100894001074A0F000000090E611F000000090E653
:1008A4005EE04408F0000000E490E68DF0000000F3
:1008B40090E65EE04404F0000000E490E7C0F090AD
:1008C400E7C4F0A3F0A3F0A3F090E7F0F090E68F74
:1008D4007440F000000090E65EE04440F000000048
:1008E4007E027F0090F800E4F0A3DFFCDEFA90E6DD
:1008F400987402F0000000E490E699F00000007E95
:10090400027F0090F800E4F0A3DFFCDEFA90E65EDC
:10091400E04480F0000000E490E69CF000000090C9
:10092400E69DF00000007F9AFE12213475280075C0
:1009340029B4754901754A907530107531B8754BF5
:1009440006754C2C12215790E67AE054FEF0E4FD33
:100954007F901220B07F647E00121BE87DFF7F42EF
:100964001220B07F647E00121BE87D827F4E12202D
:10097400B0753AFF43A020E4F53E90E782E53AF0F3
:1009840090E781E53EF012215FD20C754801753283
:1009940027753310752A051219907F887E13121A51
:1009A400BE1219907FB87E0B121ABE7F887E131276
:1009B4001ABE1213F67DFFE4FF121FFDD2F9C2F82E
:1009C400E4F54390E7C0E543F043A01053917F0260
:0209D400157597
:0E20F600EF2401FBE43EFA7D047F48021FC583
:101EEB00E53EC313FFC374809F90256BF0E4940011
:101EFB0090256AF0E53ED394004006753AFF43A067
:091F0B0020E53E700353A0DF2223
:10131100E4FC9024BDE0FEA3E02400FDEC3EFC9043
:101321002410E0FEA3E07A002400FFEA3EFEC3EDB4
:101331009FFFEC9EFE9024B2F0A3EFF09024B5E065
:101341002FF09024B4E03EF0D3EF9450EE648094FB
:101351008050129024B2E0FAA3E0FBC394B0EA6497
:1013610080947F501C9024B3E025E0FE9024B2E0ED
:101371003390256AF0A3CEF0E49024B4F0A3F0807A
:10138100337C007D14AF03AE02120BDFAC06AD0758
:101391009024B4E0FEA3E07802C333CE33CED8F973
:1013A1002DFFEC3EFE7C007D0A120BF190256AEECA
:1013B100F0A3EFF0D390256BE094FF90256AE064F1
:1013C1008094804006E4F0A374FFF0C390256AE0A6
:1013D100648094805004E4F0A3F090256AE0FEA3B9
:1013E100E0FF7C007D02120BF1C3747F9FF0E49E4D
:0413F10090256AF0E9
:0113F50022D5
:101A02007E247FBC1220F69024BDE090E7C1F090C6
:101A120024BEE090E7C2F090256BE090E7C3F0901F
:101A220024BBE0600B43A020753AFF121311800320
:101A3200121EEB902452E53AF07A247B527D017F0C
:101A420021121FE19024527402F0A37480F07A24D0
:101A52007B527D027F28121FE1E4902452F09025F0
:101A62006BE0902453F07A247B527D027F28021F80
:011A7200E192
:10102000054EE54E7002054D0545054FB5330DE5FE
:101030004DB53208121A02E4F54DF54E90E7C8E5B9
:1010400048F0A3E52BF0A3E539F0E545B52A20E506
:1010500048601124FE60080470121220D4800D1222
:1010600020E68008E4FF121E6B53A0EFE4F5452054
:10107000010302112575430190E7C0E543F0E5A0A7
:1010800030E7032008F87FAE12211E90F00074AA0A
:10109000F0A37411F0A374CCF0A374EEF0E490E626
:1010A00090F090E6917405F012112690F00074AA69
:1010B000F0A37411F0A374CCF0A374EEF0E490E606
:1010C00090F090E6917405F07FAF12211EC201E40A
:1010D000F54390E7C0E543F09024B6E06401702A40
:1010E000E536702653A0F043A0047FD07E07121A85
:1010F000BE53A0F043A00C7FD07E07121ABE53A0AF
:10110000F043A0087FD07E0780181219907FB87E28
:101110000B121ABE1219907F887E13121ABE7F8896
:061120007E13121ABE222C
:02216400D32284
:02216600D32282
:02216800D32280
:101AD50090E680E030E73A00000090E6207402F0DE
:101AE500000000E490E621F000000090E624740276
:101AF500F0000000E490E625F000000090E6267472
:101B050002F0000000E490E627F0000000D2038018
:101B150016000000E490E620F000000090E6217435
:0F1B250040F0000000C20390E6BAE0F544D3227E
:10208C0090E740E544F0E490E68AF090E68B04F0AB
:02209C00D3224D
:08214F0090E6BAE0F527D32267
:10209E0090E740E527F0E490E68AF090E68B04F0B6
:0220AE00D3223B
:02216A00D3227E
:02216C00D3227C
:02216E00D3227A
:10008000E4FFF562F56390E6B9E0244B605224F397
:10009000700302029924F870030202E024FA70034C
:1000A000020322241D60030203A0E490E68AF0907C
:1000B000E68BF090E6A0E020E1F990E68BE0E4F535
:1000C000B390E60174CAF0D20100000090E6047417
:1000D00080F00000007402F0000000E4F00203A2CF
:1000E000E490E68AF090E68BF090E6A0E020E1F95B
:1000F00090E68BE0D3943F4024E4F562744025629F
:10010000F582E434E7F583E0FF74122562F582E4BA
:100110003424F583EFF00562E562B440DF7F8A7E28
:1001200000122134902412E0FF7E0012213D902421
:1001300013E075F004A4FFAEF0122146902417E0FE
:10014000C394025013902433E090E6C07005744EBF
:10015000F08016749CF08011902433E090E6C0701B
:1001600005749FF08003749DF0902435E024FF9285
:1001700007902432E024FF9206902436E024FF9278
:1001800009902440E0753C00F53DA3E0FEA3E07C2F
:10019000002400F525EC3EF524902445E09024B69B
:1001A000F0902418E0F535E535700375350190249D
:1001B0001DE0FEA3E07C002400F529EC3EF528A319
:1001C000E0FEA3E02400F54AEC3EF549902419E056
:1001D000FEA3E02400F531EC3EF530A3E0FEA3E001
:1001E0002400F54CEC3EF54B90244DE0FFE4FDFE81
:1001F000FBFAF97801120C27A804A905AA06AB0797
:10020000902423E0FEA3E07C002400FFEC3EFEE40B
:10021000FDEB2FFFEA3EFEED39FDEC38FCC004C0DB
:1002200005C006C00790244EE0FFE4FCFDFEFBFA8B
:100230007901F8120C27D003D002D001D000EF2BA7
:10024000F542EE3AF541ED39F540EC38F53F9024B2
:1002500021E0FEA3E07C002400F52EEC3EF52D907D
:100260002447E0540FF536E4FD7F901220B090242F
:1002700013E0FCA3E0FDA3E0FEA3E0FF9024C11285
:100280000C9A9024C1A3E0FDA3E0FEA3E0FFE4FCF0
:100290009024C1120C9A0203A290E7407425F0A3A7
:1002A000740DF0A314F0A37426F0A37407F0A374E4
:1002B000EEF0A37401F0A37403F0A37453F03003C1
:1002C00005E4A3F0800690E74974FFF0000000E425
:1002D00090E68AF000000090E68B740AF00203A218
:1002E00090E6BCE0902617F07A267B177D017F50C0
:1002F000121FE17A267B177D017F50121FE190E6E5
:10030000BEE0FD7AE77B407F50121FC5E490E68A8D
:10031000F000000090E6BEE090E68BF000000002E6
:1003200003A2E490E68AF090E68BF090E6A0E0204D
:10033000E1F990E68BE0F562C29890E740E0C39463
:10034000304006E0D39436400790E740E0F4703D3B
:10035000E548703943A01090E740E0F4600AE0B44B
:10036000300FE52B64016009D20C754801C20A8088
:100370003190E740E0C394314028E0D394365022D6
:10038000E024D1F52C652B6019C20B800E90E7405C
:10039000E0B4200EE548700A43A0107548028002C0
:0303A000D322C3A2
:0103A3002237
:10203000C0E0C083C082D20F5391EF90E65D74017F
:08204000F0D082D083D0E03221
:10206000C0E0C083C0825391EF90E65D7404F0D06D
:0620700082D083D0E032B3
:10207600C0E0C083C0825391EF90E65D7402F0D059
:0620860082D083D0E0329D
:101CE100C0E0C083C08285100C85110D850D8285F1
:101CF1000C83A37402F085080E85090F850F828578
:101D01000E83A37407F05391EF90E65D7410F0D049
:061D110082D083D0E03215
:10204800C0E0C083C082D2115391EF90E65D74085E
:08205800F0D082D083D0E03209
:101C6D00C0E0C083C08290E680E030E72085080C9C
:101C7D0085090D850D82850C83A37402F085100EE8
:101C8D0085110F850F82850E83A37407F05391EF95
:0D1C9D0090E65D7420F0D082D083D0E0325C
:01217000323C
:01217100323B
:01217200323A
:012173003239
:101DB300C0E0C083C08290E65EE054FBF000000008
:101DC30090E68F7440F00000005391EF90E65FE0DF
:101DD3004404F090E65EE04404F0D082D083D0E087
:011DE30032CD
:10122500C0E0C0F0C083C082C0D075D000C000C08F
:0D12350001C002C003C004C005C006C00710
:1012420075500075510090E65EE054F7F090E6A10B
:10125200E020E1F990E780E0FF1460161460262494
:10126200D0603A2434606514606C14706E7523008B
:10127200806990E782E0F53A90E781E0F53E9024BC
:10128200BBE4F0805690E782E0902410F090E78172
:10129200E0902411F09024BB7401F0803E90E7812D
:1012A200E07005121990803390E781E0B4010512D5
:1012B2001F89802790E781E0B40305122111801B6A
:1012C20090E781E0B4FF14122104800F90E781E0DF
:1012D20024FF92088005752300D20400000090E6E6
:1012E2008DE4F05391EF90E65FE04408F090E65E03
:0412F200E04408F0DC
:1012F600D007D006D005D004D003D002D001D0004C
:0B130600D0D0D082D083D0F0D0E032F5
:012174003238
:012175003237
:101C2E00C0E0C083C08290E65EE054BFF0000000CA
:101C3E0090E6987402F000000090E699E4F000003F
:101C4E000090F800F0A3F05391EF90E65FE044406F
:0F1C5E00F090E65EE04440F0D082D083D0E032D8
:0F1B3400C0E0C083C082C0D075D000C004C0061E
:101B430090E65EE0547FF090E6A6E020E1F990E6AF
:101B53009CE0FE90E69DE07C002400F551EC3EF510
:101B63005000000090E69CE4F090E69DF05391EF66
:0E1B730090E65FE04480F090E65EE04480F093
:0D1B8100D006D004D0D0D082D083D0E03286
:012176003236
:012177003235
:012178003234
:012179003233
:01217A003232
:01217B003231
:01217C003230
:01217D00322F
:01217E00322E
:01217F00322D
:01218000322C
:01218100322B
:01218200322A
:012183003229
:012184003228
:012185003227
:012186003226
:012187003225
:012188003224
:012189003223
:01218A003222
:01218B003221
:01218C003220
:01218D00321F
:01218E00321E
:01218F00321D
:0616B8008F648C658D6655
:1016BE0053640753B0F77F0A7E00121ABEE4F56733
:1016CE00C374029567FFE564A807088002C313D8A8
:1016DE00FC30E00543800280035380FD7F0A7E00CC
:1016EE00121ABE4380017F0A7E00121ABE5380FE7C
:1016FE007F0A7E00121ABE0567E567C3940340C0D9
:10170E00E4F567C374099567FFE566AE65A807083B
:10171E008005CEC313CE13D8F930E0054380028086
:10172E00035380FD7F0A7E00121ABE4380017F0A9A
:10173E007E00121ABE5380FE7F0A7E00121ABE056C
:10174E0067E567C3940A40BB43B0087F0A7E001268
:0C175E001ABE53B0F77F0A7E00021ABECC
:09213400AD07AC06E4FF0216B889
:09213D00AD07AC067F040216B8E0
:09214600AD07AC067F010216B8DA
:1020B000902452EDF0EFC313FF7A247B527D01028E
:0220C0001FE11E
:101A730053A0F043A0087FC47E09121ABE53A0F0FE
:101A830043A00C7FC47E09121ABE53A0F043A004E6
:101A93007FC47E09121ABE53A0F043A0067FC47E02
:101AA30009121ABE53A0F043A0027FC47E09121A82
:0B1AB300BE53A0F043A0037FC47E09D7
:101ABE00EF7803C333CE33CED8F9FFEF4E6007EF86
:071ACE001F70F81E80F522D5
:05215F00D283D28422AE
:101FA800C2837F027E00121ABEC284D2837F027E61
:0D1FB80000121ABED2847F027E00021ABE03
:1020C200E4FDFC121FA80DBD00010CBC0DF5BDF610
:0120D200F21B
:0120D30022EA
:101F3D0053A0F043A0047FD07E07121ABE53A0F029
:101F4D0043A00C7FD07E07121ABE53A0F043A00809
:071F5D007FD07E07021ABECF
:100E0E009024C1E0FCA3E0FDA3E0FEA3E0FF90244C
:100E1E00B7120C9A300605C2B043A0409024B6E03B
:100E2E007003121F89300703020EFD752301E47F44
:100E3E00E87E03FDFC9024B7E0F8A3E0F9A3E0FA06
:100E4E00A3E0FBC3120C765003020EEBE523640104
:100E5E006003020EEB7FDD7E03121BE8121A029076
:100E6E0024B7E0FCA3E0FDA3E0FEA3E02418FFEE10
:100E7E0034FCFEED34FFFDEC34FFFC9024B7120C75
:100E8E009A9024B7E0FCA3A3A3E4FFFEFDEC781830
:100E9E00120C8790E7C4EFF09024B7A3E0FDA3A354
:100EAE00E4FFFEE4FC7810120C8790E7C5EFF0909B
:100EBE0024B7A3A3E0FEA3E4FFE4FDFC7808120C24
:100ECE008790E7C6EFF09024B7E0FCA3E0FDA3E027
:100EDE00FEA3E0FFE490E7C7EFF0020E3CE523B47B
:100EEE0001169024B9E0FEA3E0FF121BE8800975FD
:100EFE002301E523640160FA9024B6E07003122109
:0A0F0E0011300605D2B053A0BF2237
:1018AB008F698E688D678C66E4FFFEFDFCAB69AAC1
:1018BB0068A967A866D3120C764057000000E4FFB6
:1018CB00FEFDE566FC7818120C8790E6CEEFF00073
:1018DB000000E4FFFEE567FDE4FC7810120C879036
:1018EB00E6CFEFF0000000E4FFE568FEE4FDFC78D6
:1018FB0008120C8790E6D0EFF0000000E569FF902E
:10190B00E6D1EFF000000075BB04000000E5BB3032
:03191B00E7FB22C5
:081CAA008C668D67AB07AA06EA
:101CB200E4FDFCC3ED9567EC95665022EA90E6D010
:101CC200F0000000EB90E6D1F000000075BB0500CB
:0E1CD2000000E5BB30E7FB0DBD00010C80D526
:011CE00022E1
:101F1400AD07AC06000000ED25E0EC3390E6D0F010
:101F2400000000ED25E090E6D1F000000075BB0450
:091F3400000000E5BB30E7FB22D0
:10112600C20453A0F043A0047FD07E07121ABE5318
:10113600A0F043A00C7FD07E07121ABE53A0F04346
:10114600A0087FD07E07121ABE9024B6E0B401072D
:10115600E5367003121F3D1220C275430290E7C0A8
:10116600E543F0120E0E75430390E7C0E543F030F9
:101176000403021224E4F564F565C3E5659529E5E3
:10118600649528500D121FA80565E56570EC056489
:1011960080E8D3E53D9400E53C9400400BAD3DACC2
:1011A6003CAF31AE30121CAAD3E5259400E5249459
:1011B600004007AF25AE24121F14E4F562F563C3A1
:1011C600E563954CE562954B502C121E96E4F5644A
:1011D600F565C3E56595357480F8656498500D121C
:1011E6001FA80565E56570EA056480E60563E563A5
:1011F60070CD056280C9E4F564F565C3E565954A79
:10120600E5649549500D121FA80565E56570EC0566
:0E1216006480E8AF42AE41AD40AC3F1218AB71
:0112240022A7
:101E9600000000E53125E0E5303390E6D0F00000A3
:101EA60000E53125E090E6D1F000000075BB0400A6
:0B1EB6000000E5BB20E7033004F82229
:0D21040053A0F07526FF90E7CBE526F022F2
:1019900053A0F043A0097F287E0A121ABE53A0F07C
:1019A00043A0017F287E0A121ABE53A0F043A00371
:1019B0007F287E0A121ABE53A0F043A0027F287E21
:1019C0000A121ABE53A0F043A0067F287E0A121AFC
:1019D000BE53A0F043A0047F287E0A121ABE53A073
:1019E000F043A00C7F287E0A121ABE53A0F043A039
:1019F000087F287E0A121ABEE4F52690E7CBE5267A
:021A0000F022D2
:0D211100121A7375260390E7CBE526F02225
:101F8900121A7353A0F043A001121ABA53A0F043D6
:0F1F9900A009121ABA75260190E7CBE526F022AF
:101B8E00052FE52FB40803E4F52FE52F70047F0829
:101B9E00803DE52FB401047F0A8034E52FB40204A2
:101BAE007F02802BE52FB403047F038022E52FB440
:101BBE0004047F018019E52FB405047F058010E52C
:101BCE002FB406047F048007E52FB4070C7F0C1298
:0A1BDE001E6B7F2D7E00121ABE223E
:1020D400C202E548600B121B8E0538E53870020514
:0220E4003722A1
:1020E600E548600B0538E53870020537121B8E226D
:08215700E4F51BD2E9D2AF222E
:101D170090E678E020E6F9C2E990E678E04480F0C2
:101D2700EF25E090E679F090E678E030E0F990E68C
:101D370078E04440F090E678E020E6F990E678E035
:061D470030E1D6D2E922D2
:101D8100A90790E678E020E6F9E51B702390E67854
:101D9100E04480F0E925E090E679F08D16AF03A9E3
:101DA100077517018A188919E4F51A751B01D322E1
:021DB100C3224B
:101D4D00A90790E678E020E6F9E51B702590E67886
:101D5D00E04480F0E925E0440190E679F08D16AF7E
:101D6D0003A9077517018A188919E4F51A751B035C
:041D7D00D322C32288
:03004B00020F1889
:100F1800C0E0C083C082C085C084C086758600C01A
:100F2800D075D000C000C001C002C003C006C00711
:100F380090E678E030E206751B0602100290E6782B
:100F4800E020E10CE51B64026006751B0702100235
:100F5800E51B24FE605F14603624FE7003020FF365
:100F680024FC7003020FFF24086003021002AB1771
:100F7800AA18A919AF1A051A8F82758300120B9047
:100F880090E679F0E51A65167070751B05806B9010
:100F9800E679E0AB17AA18A919AE1A8E82758300F4
:100FA800120BBD751B02E5166401704E90E678E0E1
:100FB8004420F08045E51624FEB51A0790E678E04F
:100FC8004420F0E51614B51A0A90E678E04440F09B
:100FD800751B0090E679E0AB17AA18A919AE1A8E0E
:100FE80082758300120BBD051A800F90E678E044E5
:100FF80040F0751B008003751B005391DFD007D0AC
:1010080006D003D002D001D000D0D0D086D084D072
:0810180085D082D083D0E032C4
:101FC500121D4DE51B24FA600E146006240770F3FC
:0C1FD500D322E4F51BD322E4F51BD32239
:101FE100121D81E51B24FA600E146006240770F3AC
:0C1FF100D322E4F51BD322E4F51BD3221D
:0300000002176A7A
:0C176A00787FE4F6D8FD7581690217B1A4
:100B9000BB010CE58229F582E5833AF583E022501A
:100BA00006E92582F8E622BBFE06E92582F8E22264
:0D0BB000E58229F582E5833AF583E493227E
:100BBD00F8BB010DE58229F582E5833AF583E8F06E
:100BCD00225006E92582C8F622BBFE05E92582C81A
:020BDD00F22202
:100BDF00EF8DF0A4A8F0CF8CF0A428CE8DF0A42E2A
:020BEF00FE22E4
:100BF100C2D5EC30E709B2D5E4C39DFDE49CFCEE1F
:100C010030E715B2D5E4C39FFFE49EFE120CA6C3E4
:100C1100E49DFDE49CFC8003120CA630D507C3E4DF
:060C21009FFFE49EFE228D
:100C2700E88FF0A4CC8BF0A42CFCE98EF0A42CFC6C
:100C37008AF0EDA42CFCEA8EF0A4CDA8F08BF0A4EA
:100C47002DCC3825F0FDE98FF0A42CCD35F0FCEB49
:100C57008EF0A4FEA9F0EB8FF0A4CFC5F02ECD390E
:0F0C6700FEE43CFCEAA42DCE35F0FDE43CFC227B
:100C7600EB9FF5F0EA9E42F0E99D42F0E89C45F0D4
:010C8600224B
:100C8700E8600FECC313FCED13FDEE13FEEF13FF4B
:030C9700D8F1226F
:0C0C9A00ECF0A3EDF0A3EEF0A3EFF022CD
:101776000209D6E493A3F8E493A34003F68001F2AA
:1017860008DFF48029E493A3F85407240CC8C33374
:10179600C4540F4420C8834004F456800146F6DF43
:1017A600E4800B01020408102040809005C8E47E06
:1017B600019360BCA3FF543F30E509541FFEE49338
:1017C600A360010ECF54C025E060A840B8E493A3FF
:1017D600FAE493A3F8E493A3C8C582C8CAC583CA2A
:1017E600F0A3C8C582C8CAC583CADFE9DEE780BEE2
:0107E3000015
:100CA600BC000BBE0029EF8DF084FFADF022E4CC32
:100CB600F875F008EF2FFFEE33FEEC33FCEE9DECFB
:100CC600984005FCEE9DFE0FD5F0E9E4CEFD22ED41
:100CD600F8F5F0EE8420D21CFEADF075F008EF2F8B
:100CE600FFED33FD4007985006D5F0F222C398FD7C
:050CF6000FD5F0EA2219
:00000001FF
